:020000040800F2
:1000000060070020750700080D0300080F030008B3
:1000100013030008170300081B030008000000007A
:100020000000000000000000000000001F030008A6
:100030002103000800000000230300082503000836
:100040008F0700088F0700088F0700088F07000838
:100050008F0700088F0700088F0700088F07000828
:100060008F0700088F0700088F0700088F07000818
:100070008F0700088F0700088F0700088F07000808
:100080008F0700088F0700088F0700088F070008F8
:100090008F0700088F0700088F0700088F070008E8
:1000A0008F0700088F0700088F0700088F070008D8
:1000B0008F0700088F0700088F0700088F070008C8
:1000C0008F0700088F0700088F0700088F070008B8
:1000D0008F070008E90600088F0700088F0700084F
:1000E0008F0700088F0700088F0700088F07000898
:1000F0008F0700088F0700088F0700088F07000888
:100100008F0700088F0700088F0700088F07000877
:100110008F0700088F0700088F0700088F07000867
:100120008F0700088F0700088F0700088F07000857
:1001300000F002F800F03AF80AA090E8000C8244BF
:100140008344AAF10107DA4501D100F02FF8AFF29C
:10015000090EBAE80F0013F0010F18BFFB1A43F0A5
:10016000010318473C1300005C130000103A24BF41
:1001700078C878C1FAD8520724BF30C830C144BF0C
:1001800004680C607047000000230024002500264E
:10019000103A28BF78C1FBD8520728BF30C148BFEA
:1001A0000B6070471FB51FBD10B510BD01F034F9CD
:1001B0001146FFF7F7FF00F009F801F066F903B404
:1001C000FFF7F2FF03BC00F031FA0000002400F05A
:1001D000C3F94FF4A06001F071F84FF4E13000F082
:1001E00034FA00F091F94BE02648008800F4004012
:1001F000E8B12448067824A001F0D0F800250DE0ED
:100200002648405D2649088000BF2548001F008819
:1002100000F040000028F8D0681CC5B2B542EFDB02
:1002200020A001F0BBF800201649088028E0601CDF
:1002300084B241F2883094FBF0F100FB114028B900
:100240001AA001F0ABF823A001F0A8F8C82094FB95
:10025000F0F100FB114010B924A001F09FF81E201E
:1002600094FBF0F100FB114038B92748006808B949
:10027000012000E00020244908600A2000F0A9F9CC
:10028000B2E700001C0000200D0AC4FAB7A2CBCDD3
:10029000B5C4CFFBCFA2CEAA3A0D0A00340000208D
:1002A000043801400D0A0D0A000000000D0A414CFF
:1002B00049454E54454B204D696E6953544D333278
:1002C000BFAAB7A2B0E520B4AEBFDACAB5D1E90D76
:1002D0000A000000D5FDB5E3D4ADD7D340414C4969
:1002E000454E54454B0D0A0D0A0D0A00C7EBCAE4F2
:1002F000C8EBCAFDBEDD2CD2D4BBD8B3B5BCFCBDA7
:10030000E1CAF80D0A000000A0012142704700BFB9
:10031000FEE700BFFEE700BFFEE700BFFEE7704755
:1003200070477047704700000CB5002001900090A6
:100330006C48006840F480306A49086000BF694832
:10034000006800F4003000900198401C0190009873
:1003500018B90198B0F5A06FF1D16248006800F4B7
:10036000003010B10120009001E0002000900098C2
:10037000012843D15C48006840F010005A490860E9
:100380000846006820F0030008600846006840F056
:100390000200086053484068524948600846406877
:1003A00048600846406840F48060486008464068FD
:1003B00020F47C1048600846406840F4E81048602B
:1003C0000846006840F08070086000BF454800683B
:1003D00000F000700028F9D04248406820F0030087
:1003E000404948600846406840F00200486000BF4D
:1003F0003C48406800F00C000828F9D10CBD10B54D
:10040000FFF792FF10BD10B53648006840F00100BC
:10041000344908600846406834490840314948601A
:1004200008460068324908402E49086008460068BE
:1004300020F4802008600846406820F4FE004860F0
:100440004FF41F008860FFF7DAFF4FF00060294982
:10045000086010BD10B5002100200022214B5B6810
:1004600003F00C0121B1042906D0082928D107E0A6
:10047000214B224C236027E01F4B204C236023E0BC
:10048000184B5B6803F47010164B5B6803F4803202
:10049000022303EB904022B9194B4343174C2360CE
:1004A0000DE0104B5B6803F4003323B1144B43435E
:1004B000124C236003E0104B4343104C236003E0D5
:1004C0000D4B0E4C236000BF00BF064B5B68C3F3AF
:1004D00003130C4CE15C094B1B68CB40074C2360B9
:1004E00010BD000000100240002002400000FFF894
:1004F000FFFFF6FE08ED00E000127A000000002089
:1005000000093D000400002008B50121242000F06E
:100510006DFC4FF48070ADF8000010208DF80300E2
:1005200003208DF802006946094800F0A3F94FF452
:100530008071074800F04BFA0420ADF800006946CE
:10054000044800F097F90421024800F040FA08BD81
:10055000000801400014014010B56FF0040000F0E5
:10056000FCFE2E4800682E49B0FBF1F02D490870C2
:100570000846007800EB4001C1EBC0104FF6FF7158
:1005800001EAC0002849088010BD0146254A1278BA
:100590004A434FF0E0235A6100229A611A461269D9
:1005A00042F001021A6100BF4FF0E022106900F032
:1005B00001021AB100F48032002AF5D04FF0E02297
:1005C000126922F001024FF0E0231A6100229A61C1
:1005D00070470146144A12884A434FF0E0235A619B
:1005E00000229A611A46126942F001021A6100BFA4
:1005F0004FF0E022106900F001021AB100F48032DD
:10060000002AF5D04FF0E022126922F001024FF0EB
:10061000E0231A6100229A61704700000000002068
:1006200000127A001400002016000020014600BFCE
:10063000704700BF4B4A128802F04002002AF9D0EE
:10064000C2B2484B1B1D1A80704710B586B00446D5
:10065000012144F2040000F0C9FB424800F02AFCEA
:100660004FF40070ADF8140003208DF81600182028
:100670008DF8170005A93C4800F0FCF84FF48060A5
:10068000ADF8140004208DF8170005A9364800F0D5
:10069000F1F825208DF8000003208DF801008DF879
:1006A000020001208DF80300684600F00CFE019462
:1006B0000020ADF80800ADF80A00ADF80C00ADF868
:1006C00010000C20ADF80E0001A9264800F035FC02
:1006D000012240F22551234800F0C7FC01212148A6
:1006E00000F0B7FC06B010BD10B540F225511D4812
:1006F00000F0A0FD10B31B4800F01CFDC4B21B4865
:10070000008800F40040C8B91848008800F4804010
:1007100060B10A2C03D000201449088020E013485F
:10072000008840F400401149088019E00D2C06D1E2
:100730000E48008840F480400C49088010E00B48C7
:100740000088C0F30D000A490C5408480088401C7A
:100750000649088008460088C72801DD0020088077
:1007600010BD000000380140000801401C000020BE
:10077000340000200948804709480047FEE7FEE7AB
:10078000FEE7FEE7FEE7FEE7FEE7FEE7FEE7FEE741
:1007900004480549054A064B704700000704000855
:1007A0003101000860010020600700206003002084
:1007B0006003002010B50446CC48844208D10121D2
:1007C000042000F02DFB0021042000F029FB46E06E
:1007D000C748844208D10121082000F021FB0021F4
:1007E000082000F01DFB3AE0C248844208D10121F4
:1007F000102000F015FB0021102000F011FB2EE06E
:10080000BD48844208D10121202000F009FB0021CD
:10081000202000F005FB22E0B848844208D10121E5
:10082000402000F0FDFA0021402000F0F9FA16E027
:10083000B348844208D10121802000F0F1FA002160
:10084000802000F0EDFA0AE0AE48844207D1012191
:10085000801500F0E5FA0021A01500F0E1FA10BDC6
:1008600010B50121084600F0DBFA0021012000F05C
:10087000D7FA10BD2DE9F0410246002500260020E0
:1008800000230024002791F803C00CF00F0591F815
:1008900003C00CF0100CBCF1000F03D091F802C0A3
:1008A0004CEA050591F800C0BCF1000F31D0146886
:1008B00000202BE04FF0010C0CFA00F3B1F800C05F
:1008C0000CEA03069E4220D183004FF00F0C0CFA75
:1008D00003F7BC4305FA03FC4CEA040491F803C097
:1008E000BCF1280F06D14FF0010C0CFA00FCC2F845
:1008F00014C00AE091F803C0BCF1480F05D14FF0D5
:10090000010C0CFA00FCC2F810C0401C0828D1D31E
:100910001460B1F800C0BCF1FF0F34DD5468002052
:100920002EE000F1080C4FF0010808FA0CF3B1F8C2
:1009300000C00CEA03069E4221D183004FF00F0C49
:100940000CFA03F7BC4305FA03FC4CEA040491F8E3
:1009500003C0BCF1280F05D100F1080C08FA0CF80F
:10096000C2F8148091F803C0BCF1480F07D100F120
:10097000080C4FF0010808FA0CF8C2F81080401C6F
:100980000828CED35460BDE8F0814FF6FF71018096
:10099000022181700421C1707047024600209368D3
:1009A0000B400BB1012000E0002070470146886831
:1009B00080B2704702460020D3680B400BB1012083
:1009C00000E0002070470146C86880B270470161AE
:1009D0007047416170470AB1016100E041617047B1
:1009E000C16070474FF480320A4382618161826145
:1009F00082698269704702460020434B18684FF6AF
:100A00008073184040EA021008433F4B186070475B
:100A10003E49C8617047F0B50A4600230024002112
:100A2000002500F00046B6F1004F02D1364EF169C4
:100A300001E0354E7168C0F3034583B200F44016FF
:100A4000B6F5401F08D121F070612F4E766826F070
:100A500070662D4F7E6012E000F48016B6F5801FA0
:100A600006D1032606FA05F4A14341F0706106E0C1
:100A7000460D360103FA06F6B14341F0706122B12A
:100A8000460D360103FA06F6314300F00046B6F192
:100A9000004F02D11C4EF16101E01B4E7160F0BDB0
:100AA00030B500228B071C0F0F2303FA04F2164BFC
:100AB00008338C1053F824309343134C08348D10B2
:100AC00044F8253023468C1053F824308C07240F2B
:100AD00000FA04F423430C4C08348D1044F82530FC
:100AE00030BD0A49DC310860704700000008014051
:100AF000000C0140001001400014014000180140AA
:100B0000001C014000200140000001400000204284
:100B1000DF48006840F00100DD4908600846406891
:100B2000DC490840DA49486008460068DA4908406C
:100B3000D74908600846006820F48020086008460D
:100B4000406820F4FE0048604FF41F008860704742
:100B5000CF49096821F48031CD4A116011460968F6
:100B600021F480211160B0F5803F03D0B0F5802FD3
:100B70000ED106E0C649096841F48031C44A1160CB
:100B800007E0C349096841F4A021C14A116000E0AF
:100B900000BF00BF704710B50146002200230020AF
:100BA0004A11012A02D1BA4C236806E0022A02D176
:100BB000B74C236A01E0B64C636A01F01F020124BE
:100BC00094401C400CB1012000E0002010BD38B55D
:100BD000002000900024002500BF3120FFF7DBFF3C
:100BE00005460098401C00900098B0F5A06F01D019
:100BF000002DF2D03120FFF7CEFF08B1012400E034
:100C00000024204638BD01460020A14A106820F08B
:100C1000F80040EAC10010607047A04908607047C2
:100C2000024600209A4B586820F47C1042EA0103E7
:100C30001843974B586070479849086670470146BB
:100C40000020934A506820F003000843506070472A
:100C50008F48406800F00C007047014600208C4A25
:100C6000506820F0F00008435060704701460020B3
:100C7000874A506820F4E06008435060704701469E
:100C80000020834A506820F4605040EAC100506060
:100C9000704729B17E4A527A02437D4B5A7204E072
:100CA0007B4A527A82437A4B5A7270477B49D831D9
:100CB0000860704701460020754A506820F44040A3
:100CC0000843506070470021714A20321170704A09
:100CD00082F82010012802D004280AD104E0012162
:100CE0006B4A2032117005E00521694A20321170EB
:100CF00000E000BF00BF7047694908607047644961
:100D0000096A0143624A11627047654944390860C3
:100D1000704730B500210022002400235C4D6D682F
:100D200005F00C0121B1042905D0082923D105E0E3
:100D30005C4D056022E05B4D05601FE0544D6D6821
:100D400005F47012524D6D6805F48034022505EBF0
:100D500092421CB9544D554305600BE04C4D6D68F3
:100D600005F400351DB1504D5543056002E04D4D71
:100D70005543056002E04B4D056000BF00BF444D88
:100D80006D6805F0F0010909484D6B5C0568DD40B0
:100D900045603F4D6D6805F4E061090A434D6B5CA9
:100DA0004568DD4085603A4D6D6805F46051C90ABB
:100DB0003E4D6B5C4568DD40C560354D6D6805F4A2
:100DC0004041890B3A4D6B5CC568B5FBF3F5056195
:100DD00030BD29B12E4A526902432D4B5A6104E0BD
:100DE0002B4A526982432A4B5A61704729B1284ADB
:100DF00092690243264B9A6104E0254A9269824334
:100E0000234B9A61704729B1214AD2690243204B92
:100E1000DA6104E01E4AD26982431D4BDA617047F1
:100E200029B11B4AD2680243194BDA6004E0184A20
:100E3000D2688243164BDA60704729B1144A1269AE
:100E40000243134B1A6104E0114A12698243104BAA
:100E50001A61704712494039086070470F49C864E9
:100E600070470B49C87170470948406A40F080706C
:100E700007494862704701460020054A92680A40C7
:100E80000AB1012000E000207047014988727047D4
:100E9000001002400000FFF8FFFFF6FE0000424293
:100EA0008004424200127A0000093D001E0000202A
:100EB0002E00002010B50446FB48844209D10121D0
:100EC0008803FFF7ADFF00214FF48040FFF7A8FF34
:100ED00032E0F648844209D101214804FFF7ADFF12
:100EE00000214FF40030FFF7A8FF25E0F0488442CE
:100EF00009D101218804FFF7A0FF00214FF48020D1
:100F0000FFF79BFF18E0EB48844209D10121C80498
:100F1000FFF793FF00214FF40020FFF78EFF0BE057
:100F2000E548844208D101210805FFF786FF00212A
:100F30004FF48010FFF781FF10BD2DE9F04786B018
:100F400005460E460024A24600BFA1460027B089F0
:100F500000B100BF2F462C8A4CF6FF700440F08889
:100F600004432C82AC894EF6F3100440B0883189DA
:100F70000843718908430443AC81AC8A4FF6FF40B3
:100F80000440B0890443AC8201A8FFF7C2FEC64802
:100F9000874202D1DDF810A001E0DDF80CA0A8899D
:100FA00000F4004040B10AEBCA0000EB0A103168BF
:100FB0004900B0FBF1F807E00AEBCA0000EB0A10A9
:100FC00031688900B0FBF1F86420B8FBF0F004014F
:100FD0002009642101FB1089A88900F4004040B178
:100FE000322000EBC900B0FBF1F000F00700044331
:100FF00008E0322000EB09106421B0FBF1F000F0B2
:101000000F0004432C8106B0BDE8F0874FF4165161
:10101000016000218180C18001810C21418100217A
:101020008181704710B502460020108A4FF2FF03FD
:1010300018400B884C8823438C882343CC88234357
:101040001843108210BD0021018041808180C18041
:10105000704721B1828942F40052828104E0828982
:101060004DF6FF731A4082817047F0B503460024A5
:1010700000260025002040F66A17B94200D100BFC3
:101080001846C1F3421401F01F06012707FA06F5BE
:10109000012C01D10C3004E0022C01D1103000E011
:1010A00014301AB107682F43076002E00768AF43A6
:1010B0000760F0BD1AB1838A0B43838202E0838A02
:1010C0008B4383827047028A4FF6F0731A40028284
:1010D000028A0A430282704782894FF2FF731A40E4
:1010E000828182890A438281704721B1828942F0DC
:1010F0000202828104E082894FF6FD731A408281E8
:101100007047028A4FF6DF731A400282028A0A434E
:101110000282704721B1028A42F48042028204E0D6
:10112000028A4BF6FF731A4002827047C1F308022D
:101130008280704701468888C0F308007047818923
:1011400041F0010181817047028BD2B20283028B90
:1011500042EA012202837047028B02F47F4202833B
:10116000028B0A430283704721B1828A42F0200237
:10117000828204E0828A4FF6DF731A4082827047CF
:1011800021B1828A42F01002828204E0828A4FF604
:10119000EF731A408282704721B1828A42F00802BE
:1011A000828204E0828A4FF6F7731A408282704787
:1011B00021B1828942F40042828103E08289C2F334
:1011C0000E028281704721B1828A42F400628282DB
:1011D00004E0828A4FF2FF731A4082827047828A4B
:1011E0004FF6FB731A408282828A0A4382827047DA
:1011F00021B1828A42F00202828204E0828A4FF6A2
:10120000FD731A408282704702460020B1F5007FCC
:1012100000D100BF13880B400BB1012000E000207B
:10122000704701F40072B2F5007F00D100BFCA43DD
:101230000280704770B5024600240023002500207C
:1012400040F66A16B14200D100BFC1F3421501F069
:101250001F03012606FA03F3012D02D196893340BC
:1012600006E0022D02D1168A334001E0968A33400F
:101270000C12012606FA04F41688344013B10CB19E
:10128000012000E0002070BD10B50022002340F6D0
:101290006A14A14200D100BF0A1201249440A3B2F3
:1012A000DC43048010BD00000038014000440040D1
:1012B00000480040004C00400050004031490143CC
:1012C000314A1160704770B5002100230F22C478A5
:1012D00004B32D4C246804F4E064C4F5E064210AEE
:1012E000C1F10403CA40447804FA03F1847814403D
:1012F00021430901254C0678A155047804F01F0507
:101300000124AC4005786D11AD0005F1E025C5F86C
:10131000004109E0047804F01F050124AC401C4D95
:101320000678761145F8264070BD1A4A0A400243F5
:10133000154B1B1F1A60704739B1134A121D1268F2
:101340000243114B1B1D1A6006E00F4A121D126862
:1013500082430D4B1B1D1A607047042808D14FF0C3
:10136000E021096941F004014FF0E022116107E03A
:101370004FF0E021096921F004014FF0E0221161F2
:10138000704700000000FA050CED00E000E400E00A
:1013900080E100E080FFFF1F704700000FB40449A8
:1013A00010B503AA029800F009F810BC5DF814FB10
:1013B000180000207047704770477047074B70B5A2
:1013C0000D467B4400F011F80446284600F020F852
:1013D00010B14FF0FF3070BD204670BD6DF2FFFFC1
:1013E00001694A1C02610878704700B58FB0CDE9E9
:1013F00001310021059105497944CDE903101146D9
:10140000684600F02EF80FB000BD0000E5FFFFFFBA
:10141000007B00F080007047754600F03DF8AE4656
:1014200005006946534620F00700854618B020B5F0
:10143000FFF7AEF9BDE820404FF000064FF000077F
:101440004FF000084FF0000B21F00701AC46ACE86C
:10145000C009ACE8C009ACE8C009ACE8C0098D46D9
:1014600070472DE9F04106460024D6E90170F56881
:101470008046304603E04146B847641C3046A847E2
:101480000028F8D12046BDE8F0810446AFF3008083
:101490002046FEF794FE000000487047FC00002044
:1014A000C014000800000020340000006C01000897
:1014B000F4140008340000202C0700008801000804
:1014C00000A24A0400000000000000000102030422
:1014D00006070809000000000000000000000000EE
:1014E00000000102030401020304060708090204C4
:0414F00006080000EA
:0400000508000131BD
:00000001FF
